BL51 BANKED LINKER/LOCATER V6.22                                                        09/24/2025  17:48:50  PAGE 1


BL51 BANKED LINKER/LOCATER V6.22, INVOKED BY:
C:\KEIL_V5\C51\BIN\BL51.EXE .\Out\STARTUP.obj, .\Out\Main.obj, .\Out\pwm.obj TO .\Out\PWM_HALL_Override PRINT (.\List\PW
>> M_HALL_Override.m51) RAMSIZE (256)


MEMORY MODEL: SMALL


INPUT MODULES INCLUDED:
  .\Out\STARTUP.obj (?C_STARTUP)
  .\Out\Main.obj (MAIN)
  .\Out\pwm.obj (PWM)
  C:\KEIL_V5\C51\LIB\C51S.LIB (?C_INIT)


LINK MAP OF MODULE:  .\Out\PWM_HALL_Override (?C_STARTUP)


            TYPE    BASE      LENGTH    RELOCATION   SEGMENT NAME
            -----------------------------------------------------

            * * * * * * *   D A T A   M E M O R Y   * * * * * * *
            REG     0000H     0008H     ABSOLUTE     "REG BANK 0"
            DATA    0008H     000DH     UNIT         ?DT?MAIN
            DATA    0015H     000AH     UNIT         ?DT?PWM
            DATA    001FH     0001H     UNIT         ?DT?TEST_OVERRIDE?MAIN
            BIT     0020H.0   0000H.1   UNIT         ?BI?PWM
                    0020H.1   0000H.7                *** GAP ***
            DATA    0021H     0006H     UNIT         ?DT?_PWM_DUTY?PWM
            DATA    0027H     0001H     UNIT         ?DT?TEST_MODE?MAIN
            IDATA   0028H     0001H     UNIT         ?STACK

            * * * * * * *   C O D E   M E M O R Y   * * * * * * *
            CODE    0000H     0003H     ABSOLUTE     
            CODE    0003H     0023H     UNIT         ?C_INITSEG
            CODE    0026H     0006H     UNIT         ?PR?PWM_ISR?PWM
                    002CH     0007H                  *** GAP ***
            CODE    0033H     0003H     ABSOLUTE     
                    0036H     000DH                  *** GAP ***
            CODE    0043H     0003H     ABSOLUTE     
            CODE    0046H     00D0H     UNIT         ?PR?TEST_MODE?MAIN
            CODE    0116H     00B2H     UNIT         ?PR?TEST_OVERRIDE?MAIN
            CODE    01C8H     009AH     UNIT         ?C_C51STARTUP
            CODE    0262H     0040H     UNIT         ?PR?MAIN?MAIN
            CODE    02A2H     003DH     UNIT         ?PR?TIMER3_INTERRUPT?MAIN
            CODE    02DFH     0034H     UNIT         ?PR?_PWM_DUTY?PWM
            CODE    0313H     001DH     UNIT         ?PR?PWM_INIT?PWM



OVERLAY MAP OF MODULE:   .\Out\PWM_HALL_Override (?C_STARTUP)


SEGMENT
  +--> CALLED SEGMENT
---------------------
?C_C51STARTUP
  +--> ?PR?MAIN?MAIN
BL51 BANKED LINKER/LOCATER V6.22                                                      09/24/2025  17:48:50  PAGE 2


  +--> ?C_INITSEG

?PR?MAIN?MAIN
  +--> ?PR?_PWM_DUTY?PWM
  +--> ?PR?PWM_INIT?PWM
  +--> ?PR?TEST_OVERRIDE?MAIN



SYMBOL TABLE OF MODULE:  .\Out\PWM_HALL_Override (?C_STARTUP)

  VALUE           TYPE          NAME
  ----------------------------------

  -------         MODULE        ?C_STARTUP
  C:01C8H         SEGMENT       ?C_C51STARTUP
  I:0028H         SEGMENT       ?STACK
  C:0000H         PUBLIC        ?C_STARTUP
  D:00E0H         SYMBOL        ACC
  D:00F0H         SYMBOL        B
  D:0083H         SYMBOL        DPH
  D:0082H         SYMBOL        DPL
  N:0000H         SYMBOL        IBPSTACK
  N:0100H         SYMBOL        IBPSTACKTOP
  N:0100H         SYMBOL        IDATALEN
  C:01CBH         SYMBOL        IDATALOOP
  N:0000H         SYMBOL        PBPSTACK
  N:0100H         SYMBOL        PBPSTACKTOP
  N:0000H         SYMBOL        PDATALEN
  N:0000H         SYMBOL        PDATASTART
  N:0000H         SYMBOL        PPAGE
  N:0000H         SYMBOL        PPAGEENABLE
  D:00A0H         SYMBOL        PPAGE_SFR
  D:0081H         SYMBOL        SP
  C:01C8H         SYMBOL        STARTUP1
  N:0000H         SYMBOL        XBPSTACK
  N:0000H         SYMBOL        XBPSTACKTOP
  N:0400H         SYMBOL        XDATALEN
  C:01D6H         SYMBOL        XDATALOOP
  N:0000H         SYMBOL        XDATASTART
  C:0000H         LINE#         126
  C:01C8H         LINE#         132
  C:01CAH         LINE#         133
  C:01CBH         LINE#         134
  C:01CCH         LINE#         135
  C:01CEH         LINE#         139
  C:01D1H         LINE#         140
  C:01D3H         LINE#         144
  C:01D5H         LINE#         146
  C:01D6H         LINE#         147
  C:01D7H         LINE#         148
  C:01D8H         LINE#         149
  C:01DAH         LINE#         150
  C:01DCH         LINE#         184
  C:01DFH         LINE#         195
  -------         ENDMOD        ?C_STARTUP

BL51 BANKED LINKER/LOCATER V6.22                                                      09/24/2025  17:48:50  PAGE 3


  -------         MODULE        MAIN
  C:0000H         SYMBOL        _ICE_DUMMY_
  D:0080H         PUBLIC        P0
  D:0090H         PUBLIC        P1
  D:00A0H         PUBLIC        P2
  D:00B0H         PUBLIC        P3
  B:00A8H.7       PUBLIC        EA
  C:0046H         PUBLIC        Test_Mode
  D:00A8H         PUBLIC        IEN0
  D:00B8H         PUBLIC        IEN1
  B:0080H.1       PUBLIC        P0_1
  C:0262H         PUBLIC        main
  D:0098H         PUBLIC        SCON
  D:0088H         PUBLIC        TCON
  C:0116H         PUBLIC        Test_Override
  D:0008H         PUBLIC        gTimer3Int
  D:0009H         PUBLIC        OVRDAT
  D:000FH         PUBLIC        OVRDIS
  D:00D6H         PUBLIC        PWMAUX
  C:02A2H         PUBLIC        TIMER3_Interrupt
  D:00D0H         PUBLIC        PSW
  D:00C0H         PUBLIC        IRCON
  -------         PROC          TIMER3_INTERRUPT
  C:02A2H         LINE#         23
  C:02AFH         LINE#         25
  C:02B1H         LINE#         26
  C:02BCH         LINE#         27
  C:02C5H         LINE#         28
  C:02C7H         LINE#         29
  C:02D2H         LINE#         30
  C:02D4H         LINE#         31
  -------         ENDPROC       TIMER3_INTERRUPT
  -------         PROC          MAIN
  C:0262H         LINE#         33
  C:0262H         LINE#         34
  C:0262H         LINE#         36
  C:0267H         LINE#         37
  C:026CH         LINE#         38
  C:0271H         LINE#         39
  C:0276H         LINE#         40
  C:027BH         LINE#         41
  C:0280H         LINE#         42
  C:0285H         LINE#         43
  C:028AH         LINE#         45
  C:0299H         LINE#         46
  C:029CH         LINE#         48
  C:029FH         LINE#         50
  C:02A1H         LINE#         51
  -------         ENDPROC       MAIN
  -------         PROC          TEST_OVERRIDE
  -------         DO            
  D:001FH         SYMBOL        Loop
  -------         ENDDO         
  C:0116H         LINE#         53
  C:0116H         LINE#         54
  C:0116H         LINE#         56
  C:0119H         LINE#         57
BL51 BANKED LINKER/LOCATER V6.22                                                      09/24/2025  17:48:50  PAGE 4


  C:011CH         LINE#         58
  C:0121H         LINE#         59
  C:0126H         LINE#         61
  C:012CH         LINE#         62
  C:0132H         LINE#         64
  C:0138H         LINE#         65
  C:013EH         LINE#         67
  C:0144H         LINE#         68
  C:014AH         LINE#         70
  C:0150H         LINE#         71
  C:0156H         LINE#         73
  C:015CH         LINE#         74
  C:0162H         LINE#         76
  C:0168H         LINE#         77
  C:016EH         LINE#         78
  C:0174H         LINE#         80
  C:0177H         LINE#         82
  C:0179H         LINE#         83
  C:017CH         LINE#         84
  C:0182H         LINE#         85
  C:0188H         LINE#         86
  C:018EH         LINE#         87
  C:0199H         LINE#         88
  C:01A4H         LINE#         89
  C:01A7H         LINE#         91
  C:01A7H         LINE#         92
  C:01A7H         LINE#         94
  C:01AEH         LINE#         95
  C:01AEH         LINE#         96
  C:01B1H         LINE#         97
  C:01B7H         LINE#         98
  C:01BEH         LINE#         99
  C:01C3H         LINE#         101
  C:01C5H         LINE#         102
  C:01C5H         LINE#         103
  C:01C7H         LINE#         104
  -------         ENDPROC       TEST_OVERRIDE
  -------         PROC          TEST_MODE
  -------         DO            
  D:0027H         SYMBOL        Loop
  -------         ENDDO         
  C:0046H         LINE#         106
  C:0046H         LINE#         107
  C:0046H         LINE#         110
  C:0049H         LINE#         111
  C:004CH         LINE#         112
  C:0051H         LINE#         113
  C:0056H         LINE#         115
  C:005BH         LINE#         116
  C:0061H         LINE#         118
  C:0066H         LINE#         119
  C:006CH         LINE#         121
  C:0071H         LINE#         122
  C:0077H         LINE#         124
  C:007CH         LINE#         125
  C:0082H         LINE#         127
  C:0087H         LINE#         128
BL51 BANKED LINKER/LOCATER V6.22                                                      09/24/2025  17:48:50  PAGE 5


  C:008DH         LINE#         130
  C:0092H         LINE#         131
  C:0098H         LINE#         133
  C:009EH         LINE#         134
  C:00A4H         LINE#         135
  C:00AAH         LINE#         136
  C:00B0H         LINE#         137
  C:00B6H         LINE#         138
  C:00BCH         LINE#         140
  C:00C2H         LINE#         142
  C:00C5H         LINE#         144
  C:00C7H         LINE#         145
  C:00CAH         LINE#         146
  C:00D0H         LINE#         147
  C:00D6H         LINE#         148
  C:00DCH         LINE#         149
  C:00E7H         LINE#         150
  C:00F2H         LINE#         151
  C:00F5H         LINE#         153
  C:00F5H         LINE#         154
  C:00F5H         LINE#         155
  C:00FCH         LINE#         156
  C:00FCH         LINE#         157
  C:00FFH         LINE#         158
  C:0105H         LINE#         159
  C:010CH         LINE#         160
  C:0111H         LINE#         162
  C:0113H         LINE#         163
  C:0113H         LINE#         164
  C:0115H         LINE#         165
  -------         ENDPROC       TEST_MODE
  -------         ENDMOD        MAIN

  -------         MODULE        PWM
  C:0000H         SYMBOL        _ICE_DUMMY_
  D:00FAH         PUBLIC        PWMTBC0
  D:0080H         PUBLIC        P0
  D:00FBH         PUBLIC        PWMTBC1
  D:0090H         PUBLIC        P1
  D:00A0H         PUBLIC        P2
  D:00B0H         PUBLIC        P3
  D:00F5H         PUBLIC        PWMEN
  D:00A8H         PUBLIC        IEN0
  D:00F2H         PUBLIC        PERIODH
  D:00B8H         PUBLIC        IEN1
  D:00F1H         PUBLIC        PERIODL
  D:0015H         PUBLIC        PWM_PERIOD
  D:00EAH         PUBLIC        PWMINTF
  D:0017H         PUBLIC        gTEST
  D:0098H         PUBLIC        SCON
  D:0088H         PUBLIC        TCON
  D:00DBH         PUBLIC        DUTY0H
  D:00DDH         PUBLIC        DUTY1H
  D:00DFH         PUBLIC        DUTY2H
  C:0026H         PUBLIC        PWM_ISR
  D:00DAH         PUBLIC        DUTY0L
  D:00DCH         PUBLIC        DUTY1L
BL51 BANKED LINKER/LOCATER V6.22                                                      09/24/2025  17:48:50  PAGE 6


  D:00DEH         PUBLIC        DUTY2L
  D:0019H         PUBLIC        PWM_DUTY0
  D:001BH         PUBLIC        PWM_DUTY1
  D:001DH         PUBLIC        PWM_DUTY2
  B:0020H.0       PUBLIC        g_PwmInterrupt
  C:0313H         PUBLIC        PWM_Init
  D:00E3H         PUBLIC        PWMPOLARITY
  D:00D9H         PUBLIC        PWMOPMOD
  D:00D0H         PUBLIC        PSW
  D:00C0H         PUBLIC        IRCON
  C:02DFH         PUBLIC        _PWM_Duty
  -------         PROC          PWM_INIT
  C:0313H         LINE#         28
  C:0313H         LINE#         29
  C:0313H         LINE#         30
  C:0316H         LINE#         31
  C:0319H         LINE#         32
  C:031CH         LINE#         33
  C:031FH         LINE#         34
  C:0326H         LINE#         35
  C:032CH         LINE#         36
  C:032FH         LINE#         37
  -------         ENDPROC       PWM_INIT
  -------         PROC          _PWM_DUTY
  D:0021H         SYMBOL        nPWMD0
  D:0023H         SYMBOL        nPWMD1
  D:0025H         SYMBOL        nPWMD2
  C:02DFH         LINE#         43
  C:02EBH         LINE#         44
  C:02EBH         LINE#         45
  C:02F1H         LINE#         46
  C:02F8H         LINE#         47
  C:02FEH         LINE#         48
  C:0305H         LINE#         49
  C:030BH         LINE#         50
  C:0312H         LINE#         51
  -------         ENDPROC       _PWM_DUTY
  -------         PROC          PWM_ISR
  C:0026H         LINE#         62
  C:0026H         LINE#         64
  C:0029H         LINE#         65
  C:002BH         LINE#         66
  -------         ENDPROC       PWM_ISR
  -------         ENDMOD        PWM

*** WARNING L16: UNCALLED SEGMENT, IGNORED FOR OVERLAY PROCESS
    SEGMENT: ?PR?TEST_MODE?MAIN

Program Size: data=40.1 xdata=0 code=796
LINK/LOCATE RUN COMPLETE.  1 WARNING(S),  0 ERROR(S)
